:060000000A168A152B2BE5
:10000800F90083128712D43EA9260A128A1187168C
:100018000800F900831203138712C03EA9260A12AA
:100028008A1187160800BF2787120130A9260A12ED
:100038008A11053066200A128A11871608001430C2
:1000480066200A128A1187120330E6260A128A11DC
:10005800053066200A128A110330E6260A128A1130
:10006800013066200A128A110330E6260A128A1124
:10007800053066200A128A110230E6260A128A1111
:10008800053066200A128A112830A9260A128A1118
:10009800053066200A128A110630A9260A128A112A
:1000A800053066200A128A110130A9260A128A111F
:1000B800053066200A128A110F30A9260A128A1101
:1000C80005306628F700F70803190800FA30F80029
:1000D800F80803197128F8036C28F7036728AA3071
:1000E8000313C90083163B270A168A1500210A1232
:1000F8008A118316DC00DC0803190800253A031965
:100108008A285C08A9260A128A117628D101D20108
:10011800CD01CE0103172808840029080A168A157C
:1001280000210A168A113C230A128A11031CD028BE
:100138000313D101D20103172808840029080A16DD
:100148008A1500210A128A11BF27C300C401831629
:1001580052088312AF00831651088312AE000A308A
:10016800B000B101F8260A128A1156270A128A111C
:10017800D100A327D2000317A80A0319A90A28083F
:10018800840029080A168A1500210A168A113C23B8
:100198000A128A1103189F282808840029080A16B9
:1001A8008A1500210A128A112E3A0313031D1829F1
:1001B8004E170317A80A0319A90A0313D601D70172
:1001C80003172808840029080A168A1500210A1628
:1001D8008A113C230A128A11031C982928088400D2
:1001E80029080A168A1500210A128A11BF27C30096
:1001F800C401831657088312AF008316560883126A
:10020800AE000A30B000B101F8260A128A1156274A
:100218000A128A11D600A3270A128A11D7000317D7
:10022800A80A0319A90AE428D601D7014E16982965
:100238004E15B3294908840083170008D800840A9A
:100248000008D900C90AC90A5804031D2F293330E8
:10025800D8001930D900DA01DB0159088312C4002B
:10026800831658088312C30083165A08831243075B
:10027800840044080318440A0A168A1500210A1241
:100288008A110038831603194D29DA0A0319DB0A83
:1002980031295708560403195D295B085702031DC5
:1002A80057295A08560203185D295708DB005608D3
:1002B800DA0052085B02031D632951085A02031829
:1002C8006C295A08D1025B08AF270A128A116E29D5
:1002D800D101D201FF308316D107031CD203510A82
:1002E8000319520A03198C292030A9260A128A11E7
:1002F8006E295808840059080A168A1500210A121E
:100308008A11A9260A128A118316D80A0319D90A4A
:100318000130DA02031CDB035A0A03195B0A0319CA
:1003280076287D294D17B3293B270A168A150021FF
:100338000A128A118316DC00003A03190800643A8D
:100348000319B329023A03191C290F3A0319B329CF
:100358001A3A03191E29063A031996297628831290
:10036800C301073083164E058312C4004304831665
:1003780003195D2D4E1EC3290630D600D701490842
:10038800840083170008D300840A0008D400840A74
:100398000008D5000330C90753088312A00083164C
:1003A80054088312A100831655088312A200A301E2
:1003B800A401A501BA260A128A1183160318022A73
:1003C80053088312A000831654088312A1008316D1
:1003D80055088312A2000A168A114A230A128A11A2
:1003E800831320088316D300831221088316D400B0
:1003F800831222088316D5000330CD04CF01D00123
:100408005508540453040319AA2AD33084008313CB
:1004180000088312C300840A0008C400840A000884
:10042800C500840A0008C6000F300310C60CC50CAE
:10043800C40CC30CFF3E031D192AFF304305C70037
:10044800C801823E8316CF00831248080318013E74
:10045800FF3E8316D000FF30CF07031CD00350089F
:100468008312AF0083164F088312AE000330B0002A
:10047800B101F8262F088316D00083122E088316A0
:10048800CF0050088312A90083164F088312A800D2
:100498000A30AA00AB010A168A1113260A128A1119
:1004A80029088316D000831228088316CF00D01F8E
:1004B800612AFF30CF07031CD0034F03FF3A0A1607
:1004C8008A11D0230A128A1193270A128A114A081C
:1004D800A6004B08A7004C088B270A168A118B2503
:1004E8000A128A1183132608CA002708CB00280895
:1004F800CC004A088312A00083164B088312A1007F
:1005080083164C088312A200A3018030A4003F3058
:10051800A500BA260A128A110318982AFF308316F2
:10052800CF07031CD003AA2A831663270A128A114D
:10053800A3012030A4004130A500BA260A128A116E
:100548008316031CAA2ACF0A0319D00A5708502772
:100558000A128A11031DB32A0D3083165602831618
:1005680003130318D42A5308B6005408B7005508D3
:10057800B80056080A168A1582263008B9003108CC
:10058800BA003208BB000A168A1551250A128A11C8
:100598003608D3003708D4003808D500831603136B
:1005A800500850270A128A11031DDD2A0A308316C3
:1005B8004F0283160318032B5508540453040319D8
:1005C800732B5308B9005408BA005508BB000A1623
:1005D8008A152B240A128A1183133C083B043A0417
:1005E8003904031D732B500850270A128A11031D62
:1005F800002B023083164F028316031C742B03133F
:1006080063270A128A117030A3008930A400403091
:10061800A500BA260A128A110318142BF730152BD5
:10062800F8308316CF07031CD0034F080A168A1127
:10063800D0230A128A11932753088312AE00831617
:1006480054088312AF00831655088312B00083162E
:100658004A088312B10083164B088312B20083162E
:100668004C088312B3000A168A114D2083165308CA
:100678008312A600831654088312A7008316550810
:100688008312A80083164A088312A90083164B0810
:100698008312AA0083164C088312AB000A168A1527
:1006A80094240A128A11831329088316C800831216
:1006B80028088316C700831227088316C6008312EA
:1006C80026088316C5004808DB004708DA004608F4
:1006D800D9004508D800D301D401D501B32B83161E
:1006E80003135308B9005408BA005508BB000A168A
:1006F8008A152B240A128A1183139B27D8005308C2
:10070800BC005408BD005508BE005B088312A90050
:1007180083165A088312A800831659088312A70063
:10072800831658088312A6000A168A151B25260860
:100738008316BF00831227088316C0008312280877
:100748008316C1000A168A1539250A128A113C082F
:10075800D3003D08D4003E08D500CF01D001DC010C
:10076800DC0A5C0811270318013EC7000A168A151F
:100778000021C400840A0319C70A47080A168A1503
:100788000021C500840A0319C70A47080A168A15F2
:100798000021C600840A0319C70A47080A168A15E1
:1007A80000210A128A11BB270A128A11031DEC2B99
:1007B8008312B3270A128A11031DEC2B8312B72761
:1007C8000A128A11031DEC2B83124408831658025F
:1007D800031CF32BDC0A5C080A3A031DB52B4F08EF
:1007E8005C078312C300831650080318500ADC1BE9
:1007F800FF3E8312C4008316560883124307C500C0
:10080800831657080318570A83124407C600450879
:100818008316D102831246088316031CD203D20220
:100828005708560403191C2CFF30D107031CD203A8
:100838004D080339031D2F2C520850270A128A111C
:10084800031D292C013083165102031C352C20303E
:10085800A9260A128A11FF308316D107031CD20376
:10086800202C831603134D0803390319702C2D30DF
:100878006D2C1A270A128A1111270318013EAC00A1
:100888000A168A150021A900840A0319AC0A2C0843
:100898000A168A150021AA00840A0319AC0A2C0832
:1008A8000A168A150021AB00840A0319AC0A2C0821
:1008B8000A168A150021AC000A168A1105200A12A8
:1008C8008A112C270A128A11C2270A128A112D08A6
:1008D800303EA9260A128A118316DC035C0F3D2CD0
:1008E800500850270A128A11031D7D2C01308316E7
:1008F8004F02031C892C3030A9260A128A11FF30B6
:100908008316CF07031CD003742C831603135708D0
:1009180050270A128A11031D942C09308316560297
:10092800031C992C083083169B2C83165608DC0070
:100938007A270A128A11D602831244088316031CE6
:10094800D703D7025C080319AB2C2E30A9268316CF
:100958005C080A168A11D0230A128A1183133008F8
:10096800C2003108C3003208C4004208A600430888
:10097800A70044088B270A168A118B25831326089B
:10098800B9002708BA002808BB000A168A152B24C4
:100998000A128A119B270A128A114B2D1A270A124A
:1009A8008A1111270318013EAC000A168A15002186
:1009B800A900840A0319AC0A2C080A168A15002112
:1009C800AA00840A0319AC0A2C080A168A15002101
:1009D800AB00840A0319AC0A2C080A168A150021F0
:1009E800AC000A168A1105200A128A112C270A124D
:1009F8008A11C2270A128A112D08303EA9260A1226
:100A08008A1183165B088312B00083165A08831272
:100A1800AF00831659088312AE0083165808831254
:100A2800AD0083165C0811270318013EB4000A16AE
:100A38008A150021B100840A0319B40A34080A1679
:100A48008A150021B200840A0319B40A34080A1668
:100A58008A150021B300840A0319B40A34080A1657
:100A68008A1500210A128A11B400C2270A128A11B3
:100A7800831330088316DB0083122F088316DA00ED
:100A880083122E088316D90083122D088316D800E6
:100A9800DC035C0FD22C5708560403197628303033
:100AA800A9260A128A11FF308316D607031CD7031A
:100AB8004F2D49088400831700084D1B7F2D831292
:100AC8006F270A128A11D9000030D91BFF30DA00CB
:100AD800DB00C90AC90ADB1F882D0330CD04D809F9
:100AE800D909DA09DB09D80A0319D90A0319DA0A74
:100AF8000319DB0A882D83126F270A128A11D9007D
:100B0800DA01DB01C90AC90A57085604031D942DE6
:100B18005B085A04590458040319D60A0319D70A5A
:100B2800DC01DC0A5C0811270318013EC7000A161D
:100B38008A150021C400840A0319C70A47080A163F
:100B48008A150021C500840A0319C70A47080A162E
:100B58008A150021C600840A0319C70A47080A161D
:100B68008A1500210A128A11BB270A128A11031D4D
:100B7800CD2D8312B3270A128A11031DCD2D83129E
:100B8800B7270A128A11031DCD2D83124408831634
:100B98005802031CD42DDC0A5C080A3A031D962D62
:100BA8005C0881270A128A115708AA270A128A1193
:100BB800031DE22D560883124302831603130318FC
:100BC800E82D5608DC00002E5C087A270A128A11E4
:100BD8005708803A8312C5004408803A4502031D2D
:100BE800F82D43088316560283160318002E5C0856
:100BF800D600D701D61BD7035208510403190C2E6F
:100C08004D08033903190C2EFF30D107031CD203FA
:100C18004E1F272E5708803A8312C30083165208A6
:100C2800803A831243028316031D1C2E5108560274
:100C38000318252E5608D1025708AF270A128A1121
:100C4800272ED101D2015C0881270A128A11520885
:100C5800AA270A128A11031D352E5108831243024E
:100C680083160318432E5C087A270A128A11D102C8
:100C7800831244088316AF270A128A11452ED10120
:100C8800D201520851040319562E2030A9260A12FF
:100C98008A11FF308316D107031CD203520851046E
:100CA800031D492E4D08033903195E2E2D30A92640
:100CB8000A128A11FF308316D607031CD703560A77
:100CC8000319570A031976285B088312A8008316AC
:100CD8005A088312A700831659088312A6008316A0
:100CE80058088312A5008316560811270318013ED9
:100CF800AC000A168A150021A900840A0319AC0A57
:100D08002C080A168A150021AA00840A0319AC0ABD
:100D18002C080A168A150021AB00840A0319AC0AAC
:100D28002C080A168A150021AC000A168A1105201B
:100D38000A128A112C270A128A11C2270A128A114A
:100D48002D08303E8316DC005B2EBF27A200220E42
:100D58000F39A3000F30A3052308E6260A128A11CB
:100D68002208A3000F30A3052308E62EA21FC92ED0
:100D78002008003CA0002108031C210F003CA10012
:100D88002208031C220F803CA200A51FD82E23088E
:100D9800003CA3002408031C240F003CA4002508E1
:100DA800031C250F803CA5008030A206A506250857
:100DB8002202031D080024082102031D080023083D
:100DC80020020800A0000F30A0050708A100F0309D
:100DD800A1052008A1042108870007160130662014
:100DE8000A128A1107120800AC01AD012E1C022F4D
:100DF8003008AC070318AD0A3108AD070310B00D71
:100E0800B10D0310AF0CAE0C2F082E04031DFA2EE3
:100E18002D08AF002C08AE0008008312C300031091
:100E2800C30D0310430DEA3E84001B345B08831294
:100E3800A80083165A088312A7008316590883123C
:100E4800A600831658088312A50083165C080800BC
:100E580083132808B0002708AF002608AE0025082D
:100E6800AD000A30B100B201B301B40108000317A4
:100E7800290883120313C400831603172808831252
:100E88000313C30083160317A80A0319A90A8312B8
:100E98000313840044080800803A8312C30080309A
:100EA80043020800430883132E07C50044080318AB
:100EB800440A2F07C6004508D03E831608004A0892
:100EC8008312A00083164B088312A10083164C08D6
:100ED8008312A2000800C300840A0008C400430863
:100EE8008316D80083124408831608008312C300AF
:100EF800C401C31BC403831608008312C300C401C2
:100F0800C31BC4034408803AC50083160800A80020
:100F18005308A9005408AA005508AB000800831319
:100F28003008CA003108CB003208CC0008003C0861
:100F3800DB003B08DA003A08D900390808008312B8
:100F480046080318013EFF3E83160800803A8312C4
:100F5800450283160800031CD203D2020800460883
:100F680083165A0208004508831659020800C7006C
:100F780083165B0208008312031308003408330445
:100F8800320431040319F72FF701F70AB41BD22FE3
:100F98000310B10DB20DB30DB40DC92F34083002D2
:100FA800031DE02F33082F02031DE02F32082E0205
:100FB800031DE02F31082D02031CF12F3108AD026B
:100FC8003208031C320FAE023308031C330FAF0282
:100FD8003408031C340FB0020310B40CB30CB20C69
:100FE800B10CF70BD22F3008B0002F08AF002E0835
:080FF800AE002D08AD00080059
:1010020041347A343D34253433342E34303466342A
:101012002A3452346F3474346F34723473342A3451
:1010220045346C343D34253433342E343034663414
:101032000034850186018701DB30831685000F307D
:101042008600C030870034309900243098009030F8
:10105200831298000A128A1123200A128A1587160F
:10106200831605148514851584309F0083120608A3
:10107200FA27BF000F30BF053F08073A0030031DB3
:10108200042A0A128A110D200A128A158D30FA27B3
:10109200A8001930A9000A128A11732000300A161A
:1010A2008A1576210A128A15C930FA27A800193042
:1010B200A9007F283E08FD278600F40100300A16A9
:1010C2008A154C2383132608D1002508D00002304C
:1010D2000A128A11662000300A128A1104200A12AA
:1010E2008A152D30FA27A8001A30A900FD275108C9
:1010F200FA27AB00FD275008FA27AA000A128A1124
:1011020073200A128A1583120608FA27BF000F30CD
:10111200BF05C8300A128A1166200A128A153F08D2
:101122000F3A0319BE013F080E3A031D9A282030D8
:10113200BE003F080D3A031DA0281030BE003F0834
:101142000B3A031D5B28FD275008F80002300A16EF
:101152008A150F235108F80003300A168A150F2347
:1011620000300A128A110D200A128A156930FA27F4
:10117200A8001A30A9000A128A11732000300A1638
:101182008A1576210A128A15C930FA27A800193061
:10119200A900EF283E08FD278600F40100300A1658
:1011A2008A154C2383132608D1002508D00002306B
:1011B2000A128A11662000300A128A1104200A12C9
:1011C2008A152D30FA27A8001A30A900FD275108E8
:1011D200FA27AB00FD275008FA27AA000A128A1143
:1011E20073200A128A1583120608FA27BF000F30ED
:1011F200BF05C8300A128A1166200A128A153F08F2
:101202000F3A0319BE013F080E3A031D0A29203086
:10121200BE003F080D3A031D10291030BE003F08E2
:101222000B3A031DCB28FD275008F80000300A16A0
:101232008A150F235108F80001300A168A150F2368
:1012420000300A128A110D200A128A15A130FA27DB
:10125200A8001930A9000A128A11732000300A1658
:101262008A1576210A128A15F130FA27A800193058
:10127200A90060293E08FD278600F401F40A013026
:101282000A168A154C2383132608D3002508D20098
:1012920002300A128A11662000300A128A110420D2
:1012A2000A128A152D30FA27A8001A30A900FD2744
:1012B2005308FA27AB00FD275208FA27AA000A12A0
:1012C2008A1173200A128A1583120608FA27BF00B0
:1012D2000F30BF05C8300A128A1166200A128A1519
:1012E2003F080F3A0319BE013F080B3A031D7B2941
:1012F2004030BE003F08073A031D81298030BE00FE
:101302003F080E3A031D3B29FD275208F80006301C
:101312000A168A150F235308F80007300A168A1591
:101322000F2300300A128A110D200A128A15553035
:10133200FA27A8001A30A9000A128A117320003075
:101342000A168A1576210A128A15F130FA27A800A0
:101352001930A900D1293E08FD278600F401F40ABC
:1013620001300A168A154C2383132608D300250858
:10137200D2000A300A128A11662000300A128A113B
:1013820004200A128A152D30FA27A8001A30A90063
:10139200FD275308FA27AB00FD275208FA27AA00B7
:1013A2000A128A1173200A128A1583120608FA2772
:1013B200BF000F30BF05C8300A128A1166200A1218
:1013C2008A153F080F3A0319BE013F080B3A031D65
:1013D200EC294030BE003F08073A031DF229803055
:1013E200BE003F080E3A031DAC29FD275208F80043
:1013F20004300A168A150F235308F80005300A161E
:101402008A150F2300300A168A150B218316BB009A
:1014120001300A168A150B210A128A158316BA00A0
:10142200FD27A000FA273B080A168A15812183139B
:101432002108F1002008F00002300A168A150B215B
:101442008316BC0003300A168A150B210A128A156C
:101452008316B900FD27A000FA273C080A168A1550
:1014620081212108D5002008D40004300A168A15EB
:101472000B218316BB0005300A168A150B210A12AE
:101482008A158316BA00FD27A000FA273B080A1620
:101492008A1581212108F3002008F20006300A167D
:1014A2008A150B218316BC0007300A168A150B21F8
:1014B2000A128A158316B900FD27A000FA273C08F4
:1014C2000A168A1581212108D7002008D60000308B
:1014D2000A168A1521210A128A153E30FA27A80017
:1014E2001930A900D030AA001A30AB000A128A11B2
:1014F20073200A128A15700A0319710A0319912AB4
:101502008312540A0319550A0319912A720A0319FC
:10151200730A0319912A560A0319570A031DE92A65
:1015220000300A128A110D200A128A153E30FA275B
:10153200A8001930A9000530AA001A30AB000A121F
:101542008A11732000300A168A1576210A128A152A
:101552003E30FA27A8001930A9007D30AA001A30BF
:10156200AB000A128A11732000300A128A11042079
:101572000A128A153E30FA27A8001930A900413014
:10158200AA001A30AB000A128A1173200A128A15B5
:10159200F001F101FF308312D4000330D500F201D3
:1015A200F301FF30D6000330D700FA27BD01FE3029
:1015B2000A128A1166200A128A15BD0A14303D02E7
:1015C200031CD82A0A128A1117200A128A154D2BD7
:1015D20000300A128A110D200A128A153E30FA27AB
:1015E200A8001930A900BB30AA001A30AB000A12B9
:1015F2008A11732000300A168A1576210A128A157A
:101602000130FA27AA001030AB006030A800193070
:10161200A9007108AD007008AC00FD275508FA2733
:10162200B100FD275408FA27B0001630AE00193079
:10163200AF000A128A11732000300A128A110420A4
:101642000A128A153A30FA27AA001930AB00603024
:10165200A8001930A9007308AD007208AC00FD277C
:101662005708FA27B100FD275608FA27B0006B3059
:10167200AE001930AF000A128A1173200317BD01A0
:10168200FE300A128A1166200A128A15BD0A143027
:101692003D020318E32A412B00300A168A15212144
:1016A2000A128A153E30FA27A8001930A900D03054
:1016B200AA001A30AB006E2C0A128A1104200A12F8
:1016C2008A15A630FA27A8001A30A9000A128A1130
:1016D20073200A128A1583120608FA27BF000F30F8
:1016E200BF053F080F3A0319BE013F080E3A031D1A
:1016F2007C2B2030BE003F080D3A031D822B103098
:10170200BE003F08073A031D882B8030BE003F0809
:101712000B3A031D8E2B4030BE003E08FD2786008B
:10172200F40100300A168A154C2383132608CD00D3
:101732002508CC0002300A128A116620F401F40A4C
:1017420001300A168A154C2383132608CF00250878
:10175200CE0002300A128A11662000300A128A1163
:101762000D2070084C02A5007108031C710A4D027D
:10177200A6000A168A150B2525088316A6008312D1
:1017820026088316A700831227088316A80083124F
:10179200B101B430B2004330B30070085402A50066
:1017A2007108031C710A5502A6000A168A150B2538
:1017B2002508B4002608B5002708B6000A168A11C3
:1017C200522331088316A900831232088316AA0015
:1017D200831233088316AB000A168A118B258313F2
:1017E20026088312C900831627088312CA008316AB
:1017F20028088312CB0072084E02A5007308031C4E
:10180200730A4F02A6000A168A150B2525088316AD
:10181200A600831226088316A700831227088316C0
:10182200A8008312B1013430B2004330B300720811
:101832005602A5007308031C730A5702A6000A1673
:101842008A150B252508B4002608B5002708B6001E
:101852000A168A11522331088316A900831232080C
:101862008316AA00831233088316AB000A168A1164
:101872008B250A128A1583132608DD002708DE004D
:101882002808DF00B5300317A8001930A900FD278A
:101892004908FA27AA00FD274A08FA27AB00FD27C4
:1018A2004B08FA27AC000A128A11732000300A167C
:1018B2008A1576210A128A151930FA27A8001A30D9
:1018C200A90003135D080317AA0003135E08031798
:1018D200AB0003135F080317AC000A128A117320CE
:1018E2000A128A1583120030051E5D2B0A128A1114
:1018F20004200A128A15FA30FA27A8001A30A90021
:101902000A128A1173200A168A15DD210A128A1513
:10191200F600413A031D932C0A168A15DD210A129C
:101922008A15D9007608413A03199F2C59085A3A68
:10193200031D842C59087A3A031D842CF5010A16DA
:101942008A15DD210A128A15F6007508963E840072
:10195200760883178000F50A7608203A031DA02C2A
:101962007508963E840080010A168A15DD21F6006C
:101972000A168A15DD21D900F5010A168A15DD211C
:101982000A128A15F60075089F3E840076088000C8
:10199200F50A7608203A031DBE2C75089F3E840086
:1019A200800196300A168A1112210A128A153E08FF
:1019B200FA27B400FD273F08FA27B500FD274008A3
:1019C200FA27B60034080313A600031735080313D9
:1019D200A700031736080313A800700883125402E5
:1019E200A5007108031C710A5502A6000A168A1581
:1019F2000B252508B1002608B2002708B300B40160
:101A0200B430B5004330B6000A168A1152233108A9
:101A12008316A900831232088316AA0083123308A0
:101A22008316AB000A168A118B2583132608031727
:101A320090000313270803179100031328080317C4
:101A420092009F300A168A1112210A128A153E0844
:101A5200FA27B400FD273F08FA27B500FD27400802
:101A6200FA27B60034080313A60003173508031338
:101A7200A700031736080313A80072088312560240
:101A8200A5007308031C730A5702A6000A168A15DA
:101A92000B252508B1002608B2002708B300B401BF
:101AA2003430B5004330B6000A168A115223310889
:101AB2008316A900831232088316AA008312330800
:101AC2008316AB000A168A118B2583132608031787
:101AD200930003132708031794000313280803171E
:101AE200950000300A128A110D200A128A15E5307B
:101AF200FA27A8001A30A9000A128A1173200030AE
:101B02000A128A110D2096300A168A1112213E08F5
:101B1200C9003F08CA004008CB009F300A168A114C
:101B220012210A128A153E088316DD0083123F082D
:101B32008316DE00831240088316DF00123003177B
:101B4200A8001C30A900FD274908FA27AA00FD2792
:101B52004A08FA27AB00FD274B08FA27AC0003130B
:101B62005D080317AD0003135E080317AE000313ED
:101B72005F080317AF000A128A11732000300A129D
:101B82008A1104200A128A159130FA27A8001A3005
:101B9200A9000A128A1173200A128A15FD27051E4E
:101BA200732CD801F40100300A168A154C238313D2
:101BB2002608CD002508CC0002300A128A116620C0
:101BC2004C088316E6070318E70A83124D088316AA
:101BD200E707F401F40A01300A168A154C2383132D
:101BE2002608CF002508CE0002300A128A1166208C
:101BF2000A128A154E088316E8070318E90A8312A7
:101C02004F088316E9078312D80A19305802031CB9
:101C1200D32D831667088312A100831666088312E8
:101C2200A0001930A200A3010A168A15C02383134B
:101C320021088316E700831220088316E60067084E
:101C42008312CD00831666088312CC0083166908BE
:101C52008312A100831668088312A0001930A20023
:101C6200A3010A168A15C0230A128A1583132108B2
:101C72008316E900831220088316E800690883129C
:101C8200CF00831668088312CE00FA2710080313C8
:101C9200BC00031711080313BD0003171208031336
:101CA200BE00700883124C02A5007108031C710A61
:101CB2004D02A6000A168A150B2525088316BF00B9
:101CC200831226088316C000831227088316C100D8
:101CD2000A168A1539253C08E0003D08E1003E0855
:101CE200E200031713080313BC00031714080313BD
:101CF200BD00031715080313BE00720883124E02BB
:101D0200A5007308031C730A4F02A6000A168A155F
:101D12000B2525088316BF00831226088316C000F0
:101D2200831227088316C1000A168A1539253C0832
:101D3200E3003D08E4003E08E5008312A0014030C4
:101D4200A100A200831660088312A3008316610813
:101D52008312A400831662088312A5000A128A1154
:101D6200BA260A128A150318BB2E2030FA27B300AE
:101D7200B701D92E831660088312A000831661086A
:101D82008312A100831662088312A200A3014030CD
:101D9200A400C030A5000A128A11BA260A128A15B6
:101DA2000318D52E1030B72EFA27B301B701B70AA0
:101DB200FD27A001C030A1004030A20083166308B5
:101DC2008312A300831664088312A4008316650895
:101DD2008312A5000A128A11BA260A128A1503185A
:101DE200FE2E04305A020318FE2E8030FA27B2006B
:101DF200B8010313EB01EB0A292F83166308831240
:101E0200A000831664088312A1008316650883125A
:101E1200A200A301C030A400A5000A128A11BA26AA
:101E22000A128A150318212F04305A020318212F8F
:101E32004030FA27B200B8010313EA01EA0A292F57
:101E4200FA27B2010313EA01EB010317B801B80A3A
:101E520003136B0B332F6A0B332F8312DA0A8316A9
:101E6200EA01EB01031733083204FD278600003034
:101E72000A168A15762170084C02A5007108031C07
:101E8200710A4D02A6000A168A150B25250883162B
:101E9200A600831226088316A7008312270883163A
:101EA200A8008312B101B430B2004330B30070080D
:101EB2005402A5007108031C710A5502A6000A16F5
:101EC2008A150B252508B4002608B5002708B60098
:101ED2000A168A11522331088316A9008312320886
:101EE2008316AA00831233088316AB000A168A11DE
:101EF2008B25831326088312C900831627088312B1
:101F0200CA00831628088312CB0072084E02A5006D
:101F12007308031C730A4F02A6000A168A150B25C2
:101F220025088316A600831226088316A7008312AB
:101F320027088316A8008312B1013430B20043305F
:101F4200B30072085602A5007308031C730A5702F5
:101F5200A6000A168A150B252508B4002608B50026
:101F62002708B6000A168A11522331088316A900DF
:101F7200831232088316AA00831233088316AB0039
:101F82000A168A118B250A128A1583132608DD0088
:101F92002708DE002808DF0001300317A8000830F8
:101FA200A900FD274908FA27AA00FD274A08FA27AF
:101FB200AB00FD274B08FA27AC0003135D0803179B
:101FC200AD0003135E080317AE0003135F08031787
:101FD200AF000A128A1173200A128A15F5018312C0
:101FE2008608FA27370BCF2D380BCF2DFD27DA01C4
:0E1FF200732C831603170800831203130800D4
:10200200413430343D340034A001A101A201A301C6
:102012002C082B042A04290403194428A401A40A25
:102022000310AC1B1A28A90DAA0DAB0DAC0D10287C
:102032000310A00DA10DA20DA30D2C082802031D53
:102042002C282B082702031D2C282A082602031DF0
:102052002C2829082502031C3E282908A5022A0843
:10206200031C2A0FA6022B08031C2B0FA7022C0805
:10207200031C2C0FA80220140310AC0CAB0CAA0CEE
:10208200A90CA40B19282308A8002208A7002108DC
:10209200A6002008A50008002E30FE200A168A118C
:1020A2000310220D230DAD00AD08031D5D28AE0106
:1020B200AF01B001B10108003130FE200A168A11C9
:1020C2000310220D230DAC00AC08031958282E3042
:1020D2000B210A168A112E308400840A840A840A8B
:1020E200800131300B210A168A1131308400840AB2
:1020F200840A840A8001A801A901AA01AB017F30E8
:10210200AD022C08A03EA000AD022030AC000310AE
:10211200A80DA90DAA0DAB0D3130FE200A168A11A9
:102122002E3084000008A400840A0008A500840A56
:102132000008A600840A0008A70023082702031D3E
:10214200AC2822082602031DAC2821082502031D03
:10215200AC2820082402031CCC283130FE200A16A9
:102162008A112E30840020088002840A2108A400EB
:10217200031C240F8002840A2208A400031C240FDB
:102182008002840A2308A400031C240F8002840313
:102192008403840328142E3084000310800D840AE3
:1021A200800D840A800D840A800DAC0B8828AD1F37
:1021B200E7282D08803A9F3E031C58280310AB0CD9
:1021C200AA0CA90CA80CAD0FDF28F52820302D028F
:1021D20003185828AD080319F5280310A80DA90DF6
:1021E200AA0DAB0DAD03EB282B08B1002A08B000F5
:1021F2002908AF002808AE00080084000008A000EB
:10220200840A0008A100840A0008A200840A0008C7
:10221200A30008008400840A840A80308004840AAF
:10222200080083120313BD00BA0120210A168A1185
:102232003A08BE003B08BF003C08C00008008316F5
:10224200BF0083123A0803192B293A088400831627
:102252003F08800083163F08840083170008B800F7
:10226200C4260A168A11031C3829BF0A2B29B90170
:1022720038082D3A031D4129B901B90ABF0A452977
:1022820038082B3A03193F29B801BB01BC01BD0133
:10229200BE01BA0154293F08840000082E3A031DEA
:1022A20056293916BF0A391E4C293F0884000008F6
:1022B2003C230A168A11031C9F29B9143808083ACC
:1022C20003199B29391ABA03B80A3E088312A700D8
:1022D20083163D088312A60083163C088312A500CC
:1022E20083163B088312A4000A30A800A901AA01A0
:1022F200AB0191260A168A11831327088316BE00A2
:10230200831226088316BD00831225088316BC009B
:10231200831224088316BB003F0884008317000839
:10232200D03EBB0701300318BC070318BD070318D2
:10233200BE075329391A5329BA0A5329B8013F084B
:1023420084000008653A0319AC293F08840000089C
:10235200453A031DFB29BF0A3F08840000082D3AB5
:10236200031DB629B915BF0ABC293F08840000081D
:102372002B3A0319B4293F0884000008303A0319A4
:10238200B4293F08840000083C230A168A11031C62
:10239200F7293F0884000008D03EB800BF0A3F0872
:1023A200840000083C230A168A11031CF7290A300C
:1023B2008312A00083163808BF230A168A117027D9
:1023C2000A168A11BF0A3F08840000083C230A1635
:1023D2008A11031CF7290A308312A00083163808D9
:1023E200BF230A168A1170270A168A11B91DFB2902
:1023F200B809B80A3808BA0783123A088316031DC7
:10240200B91C082A8312840083163F0880003E0804
:102412008312AA0083163D088312A90083163C0882
:102422008312A80083163B088312A700D5260A163A
:102432008A1127088316BB00831228088316BC0062
:10244200831229088316BD003C043B04031D2E2A77
:102452008312BA01BB01BC010800BA1FA82ABA093B
:10246200BA0A3A08803A763E031C682A3B0883126D
:10247200B10083163C088312B20083163D08831212
:10248200B3000330B4001530B5005030B60052230B
:102492000A168A1164270A168A11F630BA07322AF6
:1024A2003B088312B10083163C088312B2008316E4
:1024B2003D088312B300B4012030B5004130B600AC
:1024C20052230A168A1164270A168A11BA03BA0815
:1024D200031D512AAF018030B000B101AF01B1013B
:1024E2003B088312A00083163C088312A1008316C6
:1024F2003D088312A20083162F088312A3008316BD
:1025020030088312A400831631088312A5000A1230
:102512008A11BA260A168A1183160318AE2A391CA2
:10252200A72AAC018030AD00AE01AC01AE012C088F
:102532008312A00083162D088312A10083162E0891
:102542008312A2004A230A168A11B42F952F3A0841
:10255200803A7F3E0318E42A83163B08391CC82AB6
:102562008312A00083163C088312A10083163D0843
:102572008312A2004A2320088316BB00831221087B
:102582008316BC00831222088316BD003B08831207
:10259200BA0083163C088312BB0083163D088312DF
:1025A200BC000800F0270A168A110330A900153072
:1025B200AA005030AB008B250A168A118D270A1605
:1025C2008A11F630BA070A303A02031CF82AD32AD3
:1025D200F0270A168A11A9012030AA004130AB0067
:1025E2008B250A168A118D270A168A11BA03BA0890
:1025F200031DE92AB5018030B6007F30B700FF30F5
:10260200B5007F30B600B70035088312A0008316EC
:1026120036088312A100831637088312A20083169C
:102622003B088312A30083163C088312A40083167E
:102632003D088312A5000A128A11BA260A168A11C7
:1026420083160318AE2A391C3B2BB2018030B3002B
:10265200B401B201B40132088312A0008316330818
:102662008312A100831634088312A2004A230A1699
:102672008A11B42F952FF800F7013A307802031827
:10268200482B30307802031C482BF701F70A770CED
:102692000800220821042004031908008030A20641
:1026A20008003108A8003208A9003308AA00031064
:1026B200290D2A0DAF00AF08031D632BB101B20132
:1026C200B30108003408A8003508A9003608AA009A
:1026D2000310290D2A0DB000B008031D742BB1019F
:1026E200B201B3010800AC01AD01AE013008893E70
:1026F200A800AF023308B0003608B0068030B0053B
:10270200B217B301B517B6011830AB000310AC0D08
:10271200AD0DAE0D36083302031D952B350832027E
:10272200031D952B34083102031CA32B3408B1027C
:102732003508031C350FB2023608031C360AB302F1
:102742002C140310B10DB20DB30DAB0B872B2C085B
:10275200A0002D08A1002E08A2002F08A300300817
:10276200A4000A168A1533260A168A118313200832
:10277200B1002108B2002208B3000800F800F701F6
:10278200781CC62B83122008F70703108312A00DB2
:102792000310F80CF808031DC12B77080800AF00DE
:1027A200AF1FB02CAF09AF0AF7270A168A11031C14
:1027B200482C8312C3270A168A1113260A168A1175
:1027C2003827A83E84001B300318013EBC000A16BD
:1027D2008A1500210A168A1148270A168A1500212D
:1027E2000A168A1140270A168A1500210A168A112A
:1027F20058270A168A1158260A168A1184270A1699
:102802008A1113260A168A11A4278D3E84001B30D2
:102812000318013EBF000A168A1500210A168A1102
:1028220030270A168A1500210A168A1150270A161D
:102832008A1500210A168A118316AB008B250A1607
:102842008A1108270A168A1158260A168A11AC27F5
:10285200723E84001B300318013EBC000A168A1522
:1028620000210A168A118316DB270A168A1500210F
:102872000A168A118316E2270A168A1500210A16F9
:102882008A118316AB008B250A168A111F2FFC278B
:102892000A168A11031C932C8312CB270A168A115B
:1028A20013260A168A1138278D3E84001B3003181E
:1028B200013EBC000A168A1500210A168A11482711
:1028C2000A168A1500210A168A1140270A168A1545
:1028D20000210A168A118316A8002F0827270A1634
:1028E2008A1158260A168A11D327723E84001B3099
:1028F2000318013EBF000A168A1500210A168A1122
:1029020030270A168A1500210A168A1150270A163C
:102912008A1500210A168A118316AB008B250A1626
:102922008A111F2F2F072F07723E84001B300318B6
:10293200013E8312BA000A168A1500210A168A116C
:10294200BB270A168A1500210A168A119C270A1625
:102952008A1500210A168A118316B2000800F72789
:102962000A168A11031C232D8312C3270A168A1101
:1029720013260A168A113827CF3E84001B3003180B
:10298200013EBC000A168A1500210A168A11482740
:102992000A168A1500210A168A1140270A168A1574
:1029A20000210A168A1158270A168A1158260A1671
:1029B2008A1184270A168A1113260A168A11A42755
:1029C200B43E84001B300318013EBF000A168A156C
:1029D20000210A168A1130270A168A1500210A16C2
:1029E2008A1150270A168A1500210A168A1183169F
:1029F200AB008B250A168A1108270A168A11582657
:102A02000A168A11AC27993E84001B300318013E36
:102A1200BC000A168A1500210A168A118316DB27C2
:102A22000A168A1500210A168A118316E2270A1647
:102A32008A1500210A168A118316AB008B250A1605
:102A42008A111F2FFC270A168A11031C6E2D83126E
:102A5200CB270A168A1113260A168A113827B43E82
:102A620084001B300318013EBC000A168A1500219F
:102A72000A168A1148270A168A1500210A168A118F
:102A820040270A168A1500210A168A118316A80001
:102A92002F0827270A168A1158260A168A11D327C1
:102AA200993E84001B300318013EBF000A168A15A6
:102AB20000210A168A1130270A168A1500210A16E1
:102AC2008A1150270A168A1500210A168A118316BE
:102AD200AB008B250A168A111F2F2F072F07993E4D
:102AE20084001B300318013E8312BA000A168A15AD
:102AF20000210A168A11BB270A168A1500210A1616
:102B02008A119C270A168A1500210A168A11831631
:102B1200B200080026088312B70083162708831222
:102B2200B80083162808E9270A168A11A000A0080F
:102B3200031D9F2DA601A701A801080029088312E1
:102B4200B70083162A088312B80083162B08E927D8
:102B52000A168A11A500A508031DB32DA601A70117
:102B6200A801080025087B3EA0072808A5002B081D
:102B7200A5068030A505A717AA17AB01A101A201DE
:102B8200A3010730A400261CCE2D29087A270A1695
:102B92008A1103182B0A031DA3070310A80CA70C04
:102BA200A60C0310A90DAA0DAB0DA40BC42D093060
:102BB200A400261CE42D29087A270A168A11031874
:102BC2002B0A031DA3070310A80CA70CA60C0310C5
:102BD200A30CA20CA10CA40BDA2D21088312A000D5
:102BE200831622088312A100831623088312A200EF
:102BF200831620088312A300831625088312A400DB
:102C02000A168A1533260A168A1183132008831698
:102C1200A600831221088316A700831222088316B6
:102C2200A8000800A501AB1F1D2EAA09AB09AA0A1C
:102C32000319AB0AA501A50AA91F262EA809A909ED
:102C4200A80A0319A90A0130A506A601A7012B08A3
:102C52002A0403194B2EA401A40A0310AB1B352E20
:102C6200AA0DAB0D2D2E0310A60DA70D2B082902C0
:102C7200031D3D2E2A082802031C472E2A08A802FB
:102C82002B08031CA903A90226140310AB0CAA0CDF
:102C9200A40B342E25080319532EA609A709A60A48
:102CA2000319A70A2708A9002608A8000800F701A7
:102CB200A11F622EA009A109A00A0319A10AF70106
:102CC200F70AA31F692EA209A309A20A0319A30ADC
:102CD200230822040319882EF801F80AA31B752E73
:102CE2000310A20DA30D6E2E23082102031D7B2EBD
:102CF20022082002031C842E2208A0022308031C9F
:102D0200A103A1020310A30CA20CF80B752E7708E5
:102D120003190800A009A109A00A0319A10A0800C1
:102D2200A001A101A201A301241CAB2E2808A00727
:102D3200290803110318013E031DA1072A080311E4
:102D42000318013E031DA2072B0803110318013EBD
:102D5200031DA3070310A80DA90DAA0DAB0D0310A7
:102D6200A70CA60CA50CA40C2708260425042404F1
:102D7200031D952E2308A7002208A6002108A500FE
:102D82002008A4000800F800F701F70A203A031906
:102D9200D32E0E3078020318D22E0930780203188F
:102DA200D32EF701770C0800A5018E30A600AA1FCA
:102DB200E72EA709A809A909AA09A70A0319A80AB7
:102DC2000319A90A0319AA0AA501A50A2A080319BF
:102DD200F12E0310AA0CA90CA80CA70CA60AE72E28
:102DE2002708A0002808A1002908A2002608A3009D
:102DF2002508A4000A168A1533260A168A11831397
:102E02002008A7002108A8002208A90008008313AF
:102E12002608AC002708AD002808AE002C08A60042
:102E22002D08A7002E08A8002F088312A000A101D8
:102E3200A01BA1030A30A200A301080083132608E5
:102E4200B0002708B1002808B20008008312A000D1
:102E5200A101A01BA1030A30A200A301080083164E
:102E6200A900840A83120319BF0A3F080800280830
:102E7200BA002908BB003A083A073A070800831645
:102E8200A700840A83120319BC0A3C0808008316AF
:102E9200A600840A83120319BC0A3C0808008316A0
:102EA200AA00840A83120319BF0A3F080800831686
:102EB200A8002F088312A000A101A01BA103643067
:102EC200A200A301080031088316BB008312320856
:102ED2008316BC00831233088316BD000800FA0073
:102EE20083163F088400831700087A07D03EB80093
:102EF2000800A1072A08031103182A0A031DA207C2
:102F02002B080311080083132108A9002008A80038
:102F12000A30AA00AB01080083132608BB00270869
:102F2200BC002808BD0008008312BA018030BB0033
:102F32000030BC0108008316B100840A8312031911
:102F4200BA0A3A0808002808BD002908BE003D0850
:102F52003D073D0708002008BA002108BB003A08D7
:102F62003A073A0708002008BA002108BB002208E5
:102F7200BC0008008316B000840A83120319BA0A3F
:102F82003A080800A800A901A81BA9036430AA00F6
:102F9200AB010800A800A901A81BA9030A30AA00D6
:102FA200AB0108002008BD002108BE003D083D0716
:102FB2003D070800A900840A83120319BC0A3C08D1
:102FC2000800AA00840A83120319BC0A3C080800FC
:102FD2008312B9000310380D390D831608003B081F
:102FE200A6003C08A7003D08A80008002F08803A68
:0E2FF200123E2F080800803A753E2F08080096
:10320000FE00FE1F082983137E188317000808009C
:103210008A0004088200F700831203178D008316CA
:103220008C130C1483120C08F8000800203420348E
:1032300020342034203441343334363430343D3477
:103240000034F9008712803E0A128A11A9260A1654
:103250008A158716080064008001840A0406031991
:10326000003404062C2928346E3475346C346C34E4
:1032700029340034453430343D340034253473343B
:02328000003418
:1032C000253473342534333464342534733425344D
:1032D0003434643400342034203420342034203416
:1032E00045343134383430343D340034F9008312FD
:1032F0008712943E0A128A11A9260A168A15871681
:103300000800F700831203132008F9007708F8007B
:103310007908A1007808A000080020342034203467
:10332000533465347434203461347A342034743442
:103330006F34203433343634303420342034203465
:103340000034203420342034533465347434203431
:1033500065346C34203474346F3420343134383470
:10336000303420342034203400342034203461348C
:103370007A3469346D3475347434203425343434FB
:103380002E34303466342034203420342034203439
:103390000034203420347434683465346E3420347E
:1033A00070347534733468342034443420346B34CE
:1033B0006534793420342034003483128C1AEF2998
:1033C000981CE8298316981298168312181218165A
:1033D000181DDD291A08831698129816DD291A0877
:1033E0000800203420347434683465346E3420345A
:1033F00070347534733468342034523420346B3470
:10340000653479342034203400342034203450346E
:103410006934633454347234613463346B3420342B
:103420006C3469346D34693474347334203420342A
:1034300000342034203465346C346534763461349F
:1034400074342034253434342E343034663420340B
:1034500020342034203420340034203420346134AB
:10346000643463342034763461346C3475346534B8
:103470003D34203420342534343475342034203421
:103480000034203420347534733469346E34673436
:103490002034643465346634613475346C34743487
:1034A0007334213420342034003420342034203448
:1034B0002034533465347434203465346C3420340F
:1034C00074346F34203430342034203420342034A9
:1034D00000342034203420342034533465347434A0
:1034E000203461347A34203474346F3420343034EE
:1034F00020342034203420340034203420346E34FE
:103500006F3474342034633461346C34693462341D
:10351000723461347434653464343A342034203481
:103520000034203420342034203420346D346F347F
:1035300076346534203472346F3474346F347234BA
:1035400073342034203420342034003420342034A8
:1035500020346D3461346E34753461346C3420340D
:1035600063346F346E34743472346F346C3420349A
:1035700020342034003420342034633461346C34FB
:103580006934623472346134743469346F346E3443
:103590002034643461347434613420342034003491
:1035A00049345734333446344F344C342D3450344A
:1035B0004934433454345234413443344B3420344A
:1035C000763431342E3434340034203420342034F2
:1035D000203420342034203420342034203420344B
:1035E000203420342034203420342034203420343B
:1035F0002034003420342034573461346934743436
:103600002034733465347234693461346C3420345A
:103610006434613474346134203420340034F7006D
:1036200003178D0078088C0083160C158312031382
:103630008B135530831603178D00AA308D008C1420
:10364000831203130D1E202B831603170C118312F4
:1036500003130D120800F001F101F201F301F4016E
:10366000F501F6018313493084005B300A168A1590
:103670002B21DD308400EC300A168A152B218317AC
:1036800090308400A8300A168A152B210A168A1554
:1036900083010A128A151A288312A000A301A4012B
:1036A00081309F00201C582B831203139F155A2B27
:1036B00003139F1101300A128A1166200A168A1517
:1036C0001F151F19612B1E08A20083161E088312E6
:1036D000A1002208A4002108A3002408A6002308B2
:1036E000A5000800003480343F34CD34CC343D3460
:1036F000D73423343C34123483343A34B734D1349D
:103700003834C63427343734383486343534C0340A
:10371000D6343334CC342B343234703489343034AE
:10372000E734DB342E34E5343C341E344234A234E6
:103730000D34003480343F340034203441340034BC
:10374000C834423400347A34443440341C3446346F
:103750005034C334473424347434493497341834DF
:103760004B34BC34BE344C346B346E344E3403347E
:10377000153450347934AD346034F3344934713411
:10378000F801F901230822040319E52BF701F70AD0
:103790000310A31BCF2BA20DA30DC72B0310F80DF5
:1037A000F90D23082102031DD72B22082002031C38
:1037B000E12B2208A0022308031CA103A102781414
:1037C0000310A30CA20CF70BCE2B7908A1007808EC
:1037D000A000080001340034003400340A340034FE
:1037E000003400346434003400340034E8340334EA
:1037F000003400341034273400340034A0348634CC
:1038000001340034403442340F3400348034963470
:10381000983400340034E134F53405340034CA34CB
:103820009A343B3441347A343D34253433342E34A5
:10383000303466342A345334653472346934613434
:103840006C342A3445346C343D34253433342E34CE
:1038500030346634003488240A168A150310410D6A
:10386000420D8316B800B808031D3B2CB901BA01FC
:10387000BB01BC01080088240A168A151730031002
:10388000C20CC10CC00CFF3E031D3F2C4008831628
:10389000B300BA17BB013908B4003A08B5003B08B9
:1038A000B600B7018E30B802B81F632C3808803AD2
:1038B0008F3E031C362C0310B70CB60CB50CB40CA1
:1038C000B80F5B2C712C183038020318362CB8084E
:1038D0000319712C0310B40DB50DB60DB70DB80357
:1038E000672C330803197F2CB409B509B609B70949
:1038F000B40A0319B50A0319B60A0319B70A370837
:10390000BC003608BB003508BA003408B90008000E
:1039100039088312C00083163A088312C100831647
:103920003B088312C20008002608F7002708F800A9
:103930002808F9000310780D790DA500A508031DCE
:10394000A62CA601A701A801A90108002908F700D3
:103950002A08F8002B08F9000310780D790DA4004F
:10396000A4080319A12CA717A801AA17AB01A0014D
:10397000A101A201A3017F30A5022408983EF7000F
:10398000A5021830A4000310A00DA10DA20DA30DD7
:103990002B082802031DD22C2A082702031DD22C33
:1039A00029082602031CE02C2908A6022A08031C69
:1039B0002A0FA7022B08031C2B0AA80220140310AD
:1039C000A60DA70DA80DA40BC32CA51FF42C25082C
:1039D000803A973E031CA12C0310A30CA20CA10C4F
:1039E000A00CA50FEC2C022D183025020318A12CD9
:1039F000A5080319022D0310A00DA10DA20DA30D02
:103A0000A503F82C2308A9002208A8002108A70074
:103A10002008A60008002508A0002608A100A20191
:103A20008E30A300A40133262008A5002108A6009B
:103A30002208A70008008E30A50029080319272DA9
:103A40000310A90CA80CA70CA60CA50A1D2D26086E
:103A5000A0002708A1002808A2002508A300A401AF
:103A6000332683132008A6002108A7002208A800F7
:103A700008008030C1063C08B6003D08B7003E088B
:103A8000B8003F08B9004008BA004108BB00512502
:103A90000A168A153608BC003708BD003808BE0073
:103AA000080036088312BE00831637088312BF0051
:103AB0008316380871260A168A15B500390883124C
:103AC000BE0083163A088312BF0083163B08712696
:103AD0000A168A15B400350803197C2D34083502FE
:103AE0000318842D34088312BE00831635087D2602
:103AF0000A168A15031C842D83163908B6003A0865
:103B0000B7003B08B8000800831634080319962D47
:103B10003508340203189E2D35088312BE00831623
:103B200034087D260A168A15031C9E2D8316360836
:103B3000B6003708B7003808B8000800063083160A
:103B4000B300B81BB317BB1B3317B717B801BA17AD
:103B5000BB01340835020318C62D0310B90DBA0D88
:103B6000BB0DB403340835060319C12DB303330864
:103B700007390319C12DAD2D0310B80CB70CB60CC5
:103B8000B50A350834060319E22DBC2D3508340278
:103B90000318E22D0310B60DB70DB80DB5033408A8
:103BA00035060319DE2DB303330807390319DE2D5B
:103BB000CA2D0310BB0CBA0CB90CB40A3508340674
:103BC000031DD92DB31FED2DFF30B606B706B8067D
:103BD000B60A0319B70A0319B80A331FF72DFF30C5
:103BE00078260A168A150319BA0A0319BB0AB30103
:103BF0003608B907370803110318370A031DBA0737
:103C0000380803110318380A031DBB07BB1F122E07
:103C1000FF3078260A168A150319BA0A0319BB0A57
:103C2000B301B30A39088312A00083163A0883123D
:103C3000A10083163B088312A20083163508831265
:103C4000A300831633088312A400332683132008AD
:103C50008316B600831221088316B7008312220848
:103C60008316B8000800230803193B2E22082104FC
:103C70002004031D442EA001A101A2010800A30AF3
:103C80000310A20CA10CA00CFE3022050319532E28
:103C90003F2EA30AA00A0319A10A0319A20A0310BE
:103CA000A20CA10CA00CFF30220503195D2E492E99
:103CB000A3030310A00DA10DA20DA11F582E231CBC
:103CC000A1130310A30C2308F900F801F7017708EA
:103CD000A0047808A1047908A2042408031DA217EF
:103CE00008008312C00003103F0D400D831608002A
:103CF000B906BA06BB06B90A08008312BE0219301B
:103D00003E020800AF006E302F02031C102F6430FB
:103D10008312A60083162F08B227BA003A073A0783
:103D2000A83E84001B300318013EBB000A168A150A
:103D300000210A168A158316EB270A168A15002118
:103D40000A168A158316F9270A168A1500210A16FB
:103D50008A158316A8000A308312A6006430F80082
:103D600083162F0895270A168A15B227BC003C0730
:103D70003C078D3E84001B300318013EBD000A162F
:103D80008A1500210A168A158316F2270A168A1543
:103D900000210A168A158316E4270A168A150021BF
:103DA0008316AB000A168A118B250A168A15CE27B0
:103DB0000A168A150A30F8002F089527BA003A0724
:103DC0003A07723E84001B300318013EBB000A16FE
:103DD0008A1500218316A900840A83120319BB0ADD
:103DE0003B080A168A1500218316AA00840A83124A
:103DF0000319BB0A3B080A168A1500218316AB007B
:103E00000A168A118B250A168A15CE27A901AA013E
:103E10003F30AB000A168A118B250A168A15DC2F53
:103E20000B302F02031C682F0A308312A600831662
:103E30002F08B227BA003A073A078D3E84001B309C
:103E40000318013EBB000A168A1500210A168A15BE
:103E50008316EB270A168A1500210A168A1583167F
:103E6000F9270A168A1500210A168A158316A80052
:103E70000A30F8002F089527BC003C073C07723E2B
:103E800084001B300318013EBD000A168A1500216C
:103E90000A168A158316F2270A168A1500210A16B1
:103EA0008A158316E4270A168A1500218316AB00AB
:103EB0000A168A118B250A168A15CE27A901AA018E
:103EC0003F30AB000A168A118B250A168A15DC2FA3
:103ED0002F082F072F07723E84001B300318013E66
:103EE0008312BA000A168A1500218316A600840AD6
:103EF00083120319BA0A3A080A168A150021831692
:103F0000A700840A83120319BA0A3A080A168A1506
:103F100000218316A800A901AA013F30AB000A16B0
:103F20008A118B250A168A15DC2F8312A00008300F
:103F3000A100A2012008F70007300310F70CFF3E94
:103F40000310031D9E2F220D7704A2000310A00D65
:103F500078082202031CAE2F7808A202A10B9A2F28
:103F6000220808008312A300A50126080319CC2FFC
:103F7000A401A40A0310A61BC02FA60DB92F03107D
:103F8000A50D26082302031CC92F2608A302251409
:103F90000310A60CA40BBF2F2508080083132608C6
:103FA000AC002708AD002808AE002C08A6002D089C
:103FB000A7002E08A800080083132608B0002708D1
:103FC000B1002808B2000800AA00840A831203196D
:103FD000BD0A3D080800A600840A83120319BB0A23
:103FE0003B080800A900840A83120319BD0A3D0892
:103FF0000800A700840A83120319BB0A3B080800C3
:02400E00723FFF
:00000001FF
